:100000000C945314189518951895189518951895DB
:100010001895189518951895189518951895189578
:10002000189518950C94F000189518950C94EA13EF
:100030000C940914189518950C94B20018951895FD
:1000400018951895189518954156524E4F434400EF
:10005000002001F301DC0111D80101D20101D4011A
:100060000FCC0104D60101D0010BC60101CA010465
:10007000C8010BBB0101BB0101DF010DCE0107DA95
:100080000128E10101E30101E50101E90101E701C5
:1000900001EB011BED0101EF0101F101FB00620128
:1000A000CF0545051FA20501A705049A0502A9056C
:1000B00001AB0501AD0501C8051555050163050135
:1000C0008005018305018805018B05018E0505B0BA
:1000D0000501B30501B60501B905016C0501660509
:1000E00001790501760502BC0501BF05015A05012C
:1000F000C20501C505FB62010606DB0518E2050124
:10010000E50506FB0501FF0502E70502EA05010119
:100110000620EE0501F10501F40501F805090306C5
:10012000FB0014036900000000090060008E2D0030
:100130000DE806B902E006D004E003BF09B701608C
:1001400009BF089507B9369A0895839B02C000E05D
:100150000895EBE6F0E0008111811695079516955C
:1001600007950895FA93EA932BD05FB76BB700E039
:100170000BBF04B115B1E9E6F0E020813181200F19
:10018000311F20833183EDE6F0E000810395008389
:10019000083081F4022F132F43E00E946D14EBE628
:1001A000F0E00083118300E000936D00E9E6F0E0E9
:1001B000008301836BBF5FBF0BD0E991F991189564
:1001C0006A935A934A933A932A931A930A930895F7
:1001D00009911991299139914991599169910895FC
:1001E0009A938A93FA93EA933A922A921A920A92EB
:1001F0007A93E6DF8FB79BB700E00BBF00916E00EC
:10020000002321F0EEE6F0E00A95008302E09ADF99
:100210009BBF8FBFDDDF79910990199029903990AC
:10022000E991F991899199911895F89400936E004C
:1002300078940895E199FECF30E03FBB0EBB1DBB23
:10024000E29AE19A0895E199FECF10E01FBB0EBB40
:10025000E09A0DB3089507E10E94DC1309EF0ABB91
:1002600000E00BBB0AEA07BBC498C49A00EF04BBCA
:1002700000E005BB00EB01BB00E002BB0E94980060
:10028000789401E010E00895C1D09ED30AE00E9466
:100290001501BFD0F1F700E00E9423010E94790A06
:1002A0000E94410880E090E0B8D09130E8F31091CE
:1002B000740000B30870012799F008E10E9415014D
:1002C000A8D0F1F783990CC010E008E00E94D10794
:1002D0000E94410801E000937600A6D009F085D085
:1002E00000B308700093740000918000002309F4AB
:1002F00042C09ED000FF02C001E001C000E01091AA
:100300007300011741F00093730008E475D0009169
:10031000730072D070D09AD007FF02C001E001C014
:1003200000E010916000011741F00093600009E4C3
:1003300063D00091600060D05ED088D004FF06C01A
:1003400007E45AD00E94231057D055D000917F0067
:100350000670043059F400E0009380006ED002E48F
:100360004BD078D0012F48D075D046D006E00E94FF
:1003700015014FD0F1F70E944D14002309F497CFD7
:100380000E942A14E0E5F0E00C94E81470D0F3CF5A
:100390009BD1F1CF19D3EFCF70D3EDCF04D4EBCFF6
:1003A000B3D4E9CF39D4E7CF54D4E5CF78D4E3CF71
:1003B0008AD4E1CFB6D4DFCF01E41ED0DCCF9FD406
:1003C000DACFFBD4D8CF3DD5D6CF07D3D4CFE0D228
:1003D000D2CFC3D2D0CFE5D2CECF41D5CCCF48D526
:1003E000CACF97D5C8CF05E4E8CF0E948E0D01E0B3
:1003F00000938D01089501E410E00C943C149A934D
:100400008A932BD0802F92D5002308959A938A93B4
:10041000089500916E00002308950FEFE82FF92F43
:1004200023D00083019608950091AC020023089523
:100430000E94620D00937F000895009373000E9454
:10044000970A0C943B0D00E000938000EFE7F0E08A
:100450000081089509E00C9479100E942A14902FCD
:100460000C942A14E62DF72DEF57FF4F08950E94A4
:100470003815F0D040805180642C752CEED0F1D02E
:1004800019F4F3D009F4B1DFEE240E942A14A02E4F
:100490000E942A14B02E0E942A140E942A14D2D03C
:1004A00009F4B9C0C5DFE5D007C0082F0E94D313F7
:1004B000C02E0C2DA1DFE6D00B2DBAD008F4A4C0BD
:1004C000BDD029F0C3DF07FF0FC0067069F400EB51
:1004D000A01650F400EAA01611F407E08DDF07E043
:1004E000C02EEE24E394E5CF0A2D005909F446C04E
:1004F0000051C1F1005109F445C00A9509F474C0D6
:100500000A9509F475C00A9509F477C00A9509F4AB
:1005100077C00A9551F20B5629F00250E1F00E50C7
:10052000F1F0C7CF7BD020F4082F0E94B90BC0CFC9
:10053000AED028F4082F00520E94D90BB9CF74DF37
:1005400031F071D020F4082F0E94F00BB1CF97D07A
:100550000E943D0CADCF93D00E94A90CA9CF082FCB
:10056000005CEACF8CD0E3E6F0E020813181E22F1D
:10057000F32F0995C02E012F3FDF9BCF082F0E943C
:100580007910F8CF7CD02A2F3B2F86D060E070E026
:100590000E94AE14452B462B472BF1F46FD00E94DE
:1005A000921281D083D07F704F33504560447940A0
:1005B00011F421E001C020E030E078D04F33504109
:1005C0006847794011F401E001C000E0022B032BE1
:1005D000642C752C09F441D06ED000810DDF3DD024
:1005E0006AD0C0803BD065CF4AD00E94421360CF12
:1005F000182F01E00E94A5135BCF182F00E0FACF5F
:10060000082F0E94CA1354CF0CD0EE2011F006E43C
:1006100001C001E4F1DEEFE00C944915803200E006
:1006200037C000E0E9CE803001E0900700E031C043
:1006300043D0081719072A072B0708950091800057
:1006400001300895902E0E942A14802E912A6ED493
:1006500000230895E9EAF2E008950FEF600E701E9E
:10066000089500918D0100230895009175000023E5
:100670000895882D992DA0E0B0E0089522D0082F8C
:10068000192F08958F5F9F4FAF4FBF4F089580364A
:100690009007A007B0070895442D552D569547950E
:1006A00008950E944C0DEFE6F0E0089540815181DD
:1006B000628173810895D6CE10E0080D191D20E0E7
:1006C000089521E830E008950E943815C090AB02EB
:1006D0001ED1C0DF40805180C4DF19F4C6DF09F4A9
:1006E00084DE0E942A14E02E0E942A14A02E0E946A
:1006F0002A140E942A14A6DF09F4D9C00E942A14E1
:10070000B8DF03C00E942A14BDDF0A2D91DF08F470
:10071000CEC094DFB9F30E2D005A09F46FC000511A
:1007200099F10A9509F48EC00A9509F4B5C00A95A5
:1007300009F4B8C00D5641F00250F9F00E5009F11D
:10074000005309F47BC0DECF69DF20F4DBD00E94C8
:10075000AA0BDACF9CDF28F4D5D000520E94BD0B43
:10076000D3CF62DE31F05FDF20F4CCD00E94DD0B0E
:10077000CBCFC2D00E943A0CC7CFBED00E943F0C54
:10078000C3CFC0D0005CEACF009179000023A1F470
:100790009DD0CAD09BD0D5D0BDD009F0B5CF91DFC8
:1007A000C8D0D2D00E94B311B2D06414750408F03E
:1007B000ABCF0FEF81D0F9CF7DD07CD00A2D7CDF7D
:1007C00080179107A207B20709F09ECFC0D0AE16DE
:1007D0002F0754DF18F40A19104005C05DDF041B11
:1007E000150B0F5F1F4F0E94451291D002C00FEFF3
:1007F00063D064147504D8F38AD086CF75D094D0B2
:1008000073D00F5F1F4F86D009F07ECF4A2D59DF7E
:10081000E82FF92F042D152D16950795E01BF10BE8
:10082000319687D00E231F230E94B01070D064141D
:10083000750408F069CF0FEF3FD0F9CF5DD00E946B
:100840001C0D62CF0E942A14202FCC2009F13BD02E
:100850007BD06AD04C2D50E041505040652F660F40
:10086000660B762F482359236A237B232CD0212F14
:10087000220F220B401751076207720709F044CF7D
:1008800020DF21D0009510955FD00E9412133CCF3D
:10089000F6DE0E94F01238CF0E942A14182F0E9410
:1008A000521332CF0E942A140E9490132DCFEFE0F2
:1008B0000C9449150E942A14D5DD008301E0600ED6
:1008C00000E0701E08950C2D10E03BC00E942A1419
:1008D000202F042D152D35D03AD0E823F923EE0F23
:1008E000FF1F0E1B1F0B08950E942A14202F25D0D6
:1008F0002BD0000F111F08950E942A14202F082FBB
:10090000192F08950E942A14102F082F0895662485
:1009100077240895E02FF12FA7DD20830ED014D087
:1009200016D00E171F070895E02FF12F9DDD2083AD
:10093000089503D0009510950895042D152D169552
:100940000795015010400895082319230895E42DB8
:10095000F52DF695E7953197089512D081F0A1DE37
:1009600012D00E7F1F700E33104011F006E401C04C
:1009700001E442DD0E94181101E000937500089522
:10098000D5D20023089500831183228333830895F1
:10099000F7DF31F00E945A1100E0009375002BDD63
:1009A000089534DDEDDF69F00E94861180E090E06B
:1009B00001C033DD4FDE0081118180179107C8F33C
:1009C0001ADD899199910895DBDF31F008E410E098
:1009D00020E00E9462150FDD08954AD08A3421F488
:1009E0000E942A14802F02C006E406DD843521F41B
:1009F0000E942A14802F02C006E4FEDC813421F418
:100A00000E942A14802F02C006E4F6DC873421F409
:100A10000E942A14802F02C006E4EEDC853721F400
:100A20000E942A14802F02C006E4E6DC803721F4FD
:100A30000E942A14802F02C006E4DEDC873621F4EF
:100A40000E942A14802F02C006E4D6DC823771F49B
:100A500097DF51F0D0DC06E00E941501DADCF1F7F7
:100A6000F8940C94001E02C006E4C6DC8991089537
:100A70008A930E942A14802F0895C1DC09F491C042
:100A8000092FEEE9F0E00C94E41480936100B3DCEC
:100A9000E0EAFFE031970E2F0F2BE1F700916100A4
:100AA0000E94FF100E94DC137CC0082F0E943810A7
:100AB00001E476C0809362000CEE1CE0E3E6F0E017
:100AC00000831183F5CF0E944410F2CFE6E8F1E0F5
:100AD000008100838183ECCFE6E8F1E0118180831F
:100AE000118320E0082F0E941C0DE2CFE8E8F1E01E
:100AF000EFCFE8E8F1E011818083118321E0F2CFAC
:100B0000E2E8F1E0E5CFE2E8F1E011818083D9CFBE
:100B1000E4E8F1E0DDCFE4E8F1E0F7CF482FE4E8E6
:100B2000F1E020813181E2E8F1E0008111810E9451
:100B30004D10BECF182F00E00E941A01082F0E940E
:100B4000790AB6CF11E0082F0E94E810B1CF10E06B
:100B5000FACF80DDDACF7EDDBBCF8093AB02A8CFAA
:100B600080937900A5CF80937A00A2CF80937700FD
:100B70009FCF809378009CCF80937C0099CF809307
:100B80007B0096CF80937D0093CF80937E0090CFA3
:100B9000882319F0BC9AC4988BCFBC9889CF06E4FF
:100BA0002BDC0FDF089564DFEBDEA1F1082FE6EF09
:100BB000F0E00C94E4140091610010E00E943C14F9
:100BC00001E427C00E948810F8CF0FE7F6CF0E94FB
:100BD000A500F3CF00E00E942301EFCF62DDD3DE5A
:100BE000ECCF61DD0181E9CF5EDD02811381E6CFCB
:100BF0005ADD0381E2CF01E00E94F710DECF00E072
:100C0000FBCF28DCDACF00918000D7CF06E4F4DBFD
:100C100006E4F2DB89910895F9DBB2DE81F00EDDA6
:100C200031F40ED005E5E8DB0BD006E407C00CD0AC
:100C3000F8DC092FE1DB082FDFDB01E4DDDBC1CECF
:100C40000AEA10E00C943C140E94200C802F912F93
:100C500008950E94431505DD19F407DD09F4C5DB8D
:100C60000E942A140E942A14902FA02F0FD0802FA8
:100C7000912BA22BB22B84DE31F001DD2A2F3B2FEA
:100C80000E94F50BB8DBE4E00C945415AA0FAA0BF4
:100C9000BA2F0E942A14212F220F220B0895B6DBAF
:100CA000C7DB6EDE71F0CFDB07FF03C000E0C5DB02
:100CB000CBDFB7DC092FA0DB10E0082F0E943C142B
:100CC0009ADB7FDE0895B4DB5BDEA1F0BCDB07FFBF
:100CD00010C00670043039F40ED00E94960B00E06C
:100CE0000093800006C000917F00067011F40E94FE
:100CF000970A81DB089501E000938000089540DEAB
:100D000011F08FDC78DB089593DB3ADE49F0F3DFF6
:100D10009DDB07FF05C00670043011F40E947E0AB7
:100D2000089586DB2DDE89F08EDB07FF0DC0E3DF43
:100D300000916200002319F00E94690B02C00E941A
:100D4000A20A00E00093800056DB08955FDB0E945A
:100D50002A147CDF0E942A14102F912B90DC31DEA4
:100D600008950E944315A02FB12F922F80E009C053
:100D70000E942A1410E0EA2FFB2FE80FF11F0083D6
:100D800083958917A8F3E4E00C9454150E94431549
:100D90000E942A145BDFA12F79DF902BA12BB22BAD
:100DA0000E942A14A02BB12B0E942A14B02B67DCBE
:100DB0002A2F3B2FE4E00C94541528E002E312E0C4
:100DC000D0DF28E00AE312E0CCDF28E002E412E002
:100DD000C8DF28E00AE412E0C4DF24E102E512E003
:100DE000C0DF24E106E612E0BCDF24E10AE712E0FE
:100DF000B8DF24E10EE812E0B4DF0E942A14009369
:100E0000A2020E942A140093A3020E942A140093B3
:100E1000A8029CDF1FDC008311830E942A14009328
:100E2000AB02B4DFE4EAF2E0AEDD0E942A140093E4
:100E3000AC02A6DD11F001E401C006E410E00C9460
:100E40003C14E4DA0E942A1408DB802F912B98DDF1
:100E500021F015DC0E948C10CEDAB3DD0895CFDAD4
:100E600029F0182F092F0E94D107C5DAAADD0895AD
:100E70000E9441152C970E942A14A02F0E942A1428
:100E8000802FEBDA402EAA23A9F4883020F40E94A8
:100E90002A1408830BC0A0E00E942A14EC2FFD2F17
:100EA000B0E0EA0FFB1F00831DD0B0F769DDB1F0A1
:100EB00020D013C065DD91F01CD0883018F40E816D
:100EC0009BDA0BC0A0E0EC2FFD2F3696B0E0EA0FC6
:100ED000FB1F008191DA06D0B0F78DDA2C96E6E0A0
:100EE0000C945215A395082F0695069506950A179A
:100EF000089555245A924A92692F482F50E02C2F7A
:100F00003D2F285F3F4F0C2F1D2F0E5F1F4F0C945E
:100F10004C0836DD51F00E94A407002321F001E4C3
:100F200010E00C943C1406E467DA08950E942A1439
:100F30000E942A140032104021F005E45DDA00E03E
:100F4000089559DA01E00895F8941A932A933A9390
:100F50004A935A930FEF1FEF26B3207454E030E00A
:100F60000317130799F040E238B3342738BB36B380
:100F700030742317232F11F05A9551F030E00A9561
:100F800009F41A953FE13A95F1F7E9CF00E002C084
:100F900001E000C0599149913991299119917894B2
:100FA00008950E944015602F512E80E090E0A0E04F
:100FB000B0E00091770060907800600E04E0600E71
:100FC000442407C04BD010E0E02F4DD009F050D0A2
:100FD0004394009177004016A8F3082F192F2A2F69
:100FE0003B2F44E00E94A614862F90E0A0E0B0E0E2
:100FF000800F911FA21FB31F442403C039D02ED0ED
:101000004394009178004016C8F3C39838D035D087
:1010100056D2442407C0C59852D2B695A795979545
:101020008795439410E0E62D1ED0082F24F480FF0E
:10103000F2CFC59AF1CF00FF02C0C59A01C0C59892
:101040001ED03DD2442403C018D0C19A4394451405
:10105000D8F335D2C39AE7E00C9451158F5F9F4FB8
:10106000AF4FBF4F0895F0E031974E161F07089518
:10107000880F991FAA1FBB1F0895C19820C2C19A4B
:101080001EC2C19AC3981BD21AD219D218D217D233
:10109000F4DFF5DFC39A08950E943815C02ED12ED3
:1010A000A22FB32F842E952EE62EAF84B888C39836
:1010B000042F152F0150104079D0C00ED11EA00F63
:1010C000B11F81E091E0B6FC02C0D7DFF8D171D04A
:1010D00038F077D029F090D0080D191D74D004C0D5
:1010E000612E7724680C791C4424552418C0C598B7
:1010F000E6D152D018F4002309F081E06AD020F440
:10110000012F4ED008F491E0882311F4119781E06B
:10111000992321F40FEFC00ED01E91E060D0E62D90
:10112000F72D31974E165F0678F4B69B03C05CD05E
:101130000C9301C039D0EE2021F0B69BD8CFC59AD0
:10114000D7CF55D0A1F2FBCFB69B02C04DD003C084
:1011500080950C9108230C93EE2021F0B69B04C0DF
:10116000C59A03C044D0E1F7C598B7FC10C087DF2B
:10117000A6D10FE3B0220A2D0B2949F080E002C06E
:101180007CDF839590E08A159B05D0F3C19A97D1B7
:10119000C39AE1E10C944915880F990F00917A00E8
:1011A00010E0401651060895082F29C043E00C9422
:1011B0006D1400E00C9300917A00109179000117F2
:1011C0000895012F08C0609079007724600E711E89
:1011D00008950091790010917A000117089501E0B7
:1011E000400E00E0501E08950C91082B0895EC2D40
:1011F000FD2D008109230895012F10E00895009529
:101200001C9110231C9308950E943915802E912E55
:10121000A22FB32FA42EB52EC62ED72EC3980FEF14
:10122000A00EB01E0A2D1B2DC1DF402E512E6FD0F7
:1012300011F0840C911E6ED011F0A40DB51D81E04B
:1012400091E06BD053D166D011F000E00C9367D0E1
:1012500038F0B7DF29F0D0DF0A0D1B1DB4DF04C062
:10126000612E77246A0C7B1C442455241CC0C5982D
:101270003DD192DF18F4002309F081E0AADF20F4C9
:10128000012F8EDF08F491E0992331F440D019F05A
:101290000FEF800E901E91E0882321F43BD009F0DF
:1012A000119781E09CDF4614570434D068F431F084
:1012B000B69B03C099DF0C9301C076DF28D0C1F242
:1012C0002FD0A9F2C59AD4CF41F0B69B02C08CDFD3
:1012D00003C080950C9108230C9319D029F020D0DD
:1012E00011F0C59A01C0C598C19A00D1FFD00C2D4C
:1012F0000D2941F080E011D0839590E08C159D057B
:10130000D0F3C19AF3D0C39AEEE00C944A15082D9D
:10131000092908950A2F0B2B0895C198E7C04BCFD8
:10132000E82DF92D0081092308950E943D15A02F75
:10133000B12F422E532E842F952F0FEF400E501EAB
:10134000042D152D33DFA00FB11F66246394E5DF54
:10135000CDD02FDF58F035DF49F04EDF040D151DDD
:10136000809079009924800E911E04C0812E9924CA
:10137000840C951C4424552410C0062D40DFB6D0A3
:10138000660C0CDF20F4002311F0662463946620C1
:1013900019F411976624639422DF4814590430F439
:1013A000B69BEBCF0C9106290C93E9CFB69B03C0FB
:1013B0000C91062903C060940C9106210C93C19AEC
:1013C00095D094D0082F092B21F0A0E009D0F0F39C
:1013D000C19A8CD000E000938000EAE00C944E1596
:1013E000C19884D0A395B0E0A817B90708950E94CA
:1013F0003D15A02FB12F842F952F21503040C39839
:10140000022F132FD3DEA00FB11F442443945C900E
:1014100000917900002319F401E000938B017FDF34
:1014200038F0CFDE29F0E8DE020F131FCCDE04C057
:10143000612E7724620E731E00918B01002311F040
:10144000622E732E6ADF52D08824992418C0C59862
:101450004DD0440CBEDE50F4CFDE8016910630F441
:1014600000918B01002311F444244394442019F487
:101470005E904424439401E0800E00E0901E8614A8
:10148000970428F4042D052111F3C59AE1CF0C919E
:10149000042111F0C59A01C0C598C19A27D026D061
:1014A000082F092B21F0A0E09BDFF0F3C19A1ED09A
:1014B000C39A00E000938B01EAE00C944E15009172
:1014C0008A010023C79A11F4C798089501E001C06A
:1014D000039510918A010117D8F3C79801E001C064
:1014E000039510918A010117D8F30895C79AC798F8
:1014F00008951FEF101B10938A01089503D099F0EF
:1015000009D011C0E9D400E000938E0100918D0153
:101510000023089535D400E000938D01089503D091
:1015200004E00C94150110E009E00C94D10701D0FF
:1015300004C010E008E00C94D107ECD301E0009364
:101540008E01E9CF269710E062D071F5F2DF68D006
:1015500000E1088300917D00098300917E000A83E9
:1015600000E010E023D036D02DD05ED001E077D05F
:1015700065D078D059D000E0088360D06BD076D0A9
:1015800011F078D0E1F74CD05CD023D0CCDF63D021
:101590006DD011F06FD0E1F743D00CD01BD06FD0DD
:1015A0000C81077F13D0C9DF269608951A930A93FA
:1015B00070D07FD008E0088367D060E045E073D04A
:1015C00000E008950D810A830C810860098308E119
:1015D000088300E05AD05DD06CC00AE053D061E0CF
:1015E00040E161D000E003D6088301E000D6098322
:1015F00001E008951A930A9360E060D0295F57D004
:1016000043D060E045E15DD0295F3F4F51C00CE021
:1016100039D061E047D00B810023089557D0802F47
:1016200010E00BE00C94D10710E00CE00C94D10713
:1016300045D02C5F3CD000E00883098326D060E0D1
:10164000089500E1088300917C00098300917B00EC
:101650000A83089527D000E10C9415010DE008835A
:1016600000E0089541E02DD02B5F21C02BD2067001
:101670000430089500916E000023089509830D81C0
:101680000A8308950E94D10700E010E01A930A939C
:10169000089560E045E150E02C2F3D2F2B5F3F4F38
:1016A0000C2F089541E050E02C2F3D2F2B5F3F4F32
:1016B0000C2F1D2F0E5F1F4F0C944C0845E001C0EE
:1016C00040E250E02C2F3D2F08959A938A9326975D
:1016D0000895269710E09BDF39F5009180000023E4
:1016E00031F027DFB8DFC2DF11F0C4DFE1F79CDFA4
:1016F00001E0B5DFA3DFB6DF93DFA3DF00E010E09A
:1017000055DF68DF5FDF90DF00E0088397DFA2DF4F
:10171000ADDF11F0AFDFE1F783DF4CDF5BDFAFDF81
:101720000C81077F53DF09DF26960895EBDE09F071
:10173000F1DE07D0F4DE9ADF11F09CDFE1F706D08E
:10174000F7CE00E28AC404D02B5FB1DF00E485C489
:1017500040E1B7CF06D00AD0108308950B2FF4D202
:1017600010E0E02FF0E00895E82FF0E0E157FE4FA1
:101770000895F7DFFBDF008108950ED0812F09D097
:101780000A2FBDD30DD010D080838991A9910895DF
:1017900010810DD010E10895AA938A93A02F089587
:1017A000EA2FF0E00895F0E0E155FE4F089500E1E2
:1017B000C8C3D7DFF9DF00810895EEDF812F412F05
:1017C00008D0FBD30A2FC0D2CCDF07D0DDCF0091E9
:1017D000A30210E020E030E00895E355FD4F0895A6
:1017E000B3D2BFDFFADF0081089527D000831183D1
:1017F000228333830895F0E01AD01FD014D0F7D39A
:10180000C4D31091AE0117D01091AD010EE199C370
:10181000232F220F220B11D00083318322832383B5
:101820000895E4EAF2E0108116500EE18AC3808147
:1018300091810697192F0FE184C3E5E6F0E0089542
:10184000FCDF13C07ED3EFE6F0E00FD03F700F3324
:101850001045204439400895E4DFE4EAF2E00081D5
:10186000118106501040E7DF90C300811181228171
:1018700033810895422FAEDFA0C3ACDF8CC38CDF71
:10188000822F95DF1A2F01E14BD002E15AD314E0E9
:1018900003E157D312E004E1D5DF11F421E001C0E8
:1018A00020E041D011F401E001C000E0022B032B45
:1018B00010E149F042D000E222D313E10FE11FD33F
:1018C00014E10FE108C03ED00DE119D313E10CE1A2
:1018D00016D314E10CE113D3BEDEB5DF11F421E021
:1018E00001C020E020D011F401E001C000E0022B93
:1018F000032B11F01FE101C01CE100E135D300E131
:1019000068DF49D3027011F0B5DE39F78991A991EA
:10191000089500E129D310E10091A202F0C20FE185
:1019200010D3182F089530E0408151816281738176
:101930004F33504168477940089502E2E0D211E107
:1019400001E204C00FE1DBD211E10EE1D8D212E1D5
:1019500008958A93802F00E1E3DF01E1F2D211E0E4
:1019600002E170DF11F421E001C020E0DCDF11F4BE
:1019700001E001C000E0022B032B10E129F0DDDFC4
:101980000FE1BDD210E204C0DDDF0CE1B8D21DE1F1
:10199000C0DF8991089516D011D000E00883098333
:1019A0009A838B834BDE12D000E048DE0FD01C817F
:1019B0000D812896899199910895098310E00AE094
:1019C0000C94D1079A938A93289703C079DE2A5FF3
:1019D0004CCE802F912F0895F5DF04E908830CE0A9
:1019E000098300E03AD3EADF01E028DEEFDF9883E5
:1019F000898302E023DEACDE2A5F14D006D02A5FA2
:101A0000A4DED5CF0AE00E94D1073EDE61E058CEC9
:101A10009FDE2C5F07C09CDE2B5F04C052DE07D028
:101A20000B5F02C005D00E5F1F4F0C944C082E5F59
:101A30003F4F0C2F1D2F08950E9443152697A02F6E
:101A4000B12F822F823098F4EBDD082F00610883DC
:101A5000B983AA8300E010E0A9DDBCDD10DE2C8193
:101A600008E010E0482F0E947314022BAFDD269689
:101A7000E4E00C9454152697D3DD9CDDABDD08D053
:101A8000007E09830D8107700A83A3DD26960895E1
:101A900008E108830C81089528970E94410810E00E
:101AA00001E00E94D10700E0C9DD0ADE0AD00A5F2A
:101AB0001F4F0E944C08388129811A810B8128967A
:101AC0000895B5CF8A93249780B38870A9DDC6DDC9
:101AD000B5DDAEDD9DDF00B30870802B11F000E0B6
:101AE00003C00B810F7100682496899108958A9331
:101AF0002A9795DDB3DD10E07DDD0DE108838823B5
:101B00000E8111F0006801C00F7704D079DD2A96AC
:101B10008991089509830F810A8308950E944115D0
:101B20002A978399B7C000918E01002339F410E001
:101B300069DF295F77DF3F8108856ADECAD0A0E0D0
:101B40001A2FCAD0EA2F11DE0083A395A032C0F36A
:101B50000091A302003620F03ADE1DD200938C01E2
:101B6000C3D0C5D08081A8E080FBB6F4C2D011F408
:101B700000E0BDDF142D00E1F7D1BBD009F4A9D0FE
:101B800000917600013031F4B4D021F400E00093EC
:101B9000760006C0A0D001C000E0E42D04DE008382
:101BA00086954394AA9501F793959830D0F2AAD0E0
:101BB000C1F099D012C09BD080A1A0E080FB46F478
:101BC0000B2F07DEE8D1E42DF0E007DE008343941D
:101BD00094D011F084D090F3939560D00917104001
:101BE00054F71EDD08E03BDD10E004DD08E167D0BE
:101BF00007DD16DD33DD10E0FDDC0DE160D000DD3A
:101C000073D075D08085A0E080FB5EF4142D81DE5A
:101C1000242D30E0205C3F4FE22FF32FC5DD008301
:101C200004C020E0042D43D0208386955524E09104
:101C3000AC02F0E0E056F0404E165F0619F0439417
:101C40004FD010F393959830E0F25CD0C9F04BD0B0
:101C500013C04DD084A9A0E080FB4EF40B2FB9DD5A
:101C60009AD1E42DF0E0E551FD4F0083439445D037
:101C700011F035D088F3939511D0091710404CF727
:101C8000CFDCECDC10E0B6DC0DE108830E810F7BCD
:101C900041DFB6DC2A96E6E00C9452150091AC02C6
:101CA00010E00056104048E050E00C94921410E010
:101CB000005C1F4FE02FF12FE155FE4F0895088380
:101CC0000E81006427CF00E012DF00912F02002375
:101CD000089501E00CCF10E10091A20210C1B3956C
:101CE000A395A8300895B0E6442490E00895E92F24
:101CF0000DC00091A2024016089586950091AC0295
:101D0000B01708950091AC0200230895F0E0EE5C56
:101D1000FD4F08958A932A97839913C010E072DECD
:101D2000D0DE095F1F4F0E944C083A810B8170DDA5
:101D3000D0DF8EE1182FD0DF17DD0083839580324E
:101D4000C8F32A968991089530E0005610E040E0EB
:101D5000E42FDCDF50A120E050FB0EF413955695E4
:101D6000301721F0339523952830B0F34395202F79
:101D7000269526952695241758F71A95012F08952C
:101D80000E94431526978399A0C00091A3020036B4
:101D900020F040918C011BDD10D180E0A0E000DD3F
:101DA000B6DF9089B8E090FB76F4E82FFCDC108178
:101DB000FEDC8ED011F400E09ADE10E1082F9FD0F7
:101DC00087D009F486DF96958395BA9561F788DF09
:101DD00030F398DFD9F0B0E6A0E014C0E1DCE658BB
:101DE000FD4F908180E090FB36F4B8DCF6DC40815A
:101DF0000B2FF0DCE2D06AD021F0B39583958830C8
:101E000090F3A3954BDF0A17104044F709DC0DE06F
:101E1000D2DBE0DB0DE13DDE006430DCDADB80E0CC
:101E2000A0E0BEDC74DF908DB8E090FB2EF4082FAC
:101E30003EDFAEDC082F63D096958395BA95A9F75F
:101E40004FDF78F35FDFE1F0B0E6A0E015C0A8DC7B
:101E5000E257FD4F908180E090FB3EF47FDCE5513E
:101E6000FD4F40810B2FB6DCA8D030D021F0B395C8
:101E70008395883088F3A39511DF0A1710403CF74B
:101E800080E072DC85DC082FABD083958031C8F30D
:101E900080E16ADC1081082F54D083958032C8F32A
:101EA000E5E6A9DCBDDB0DE086DB94DB0DE1F1DDD1
:101EB0000F7BE4DB8EDB07DF41F043DC10E08DDBE2
:101EC000BDDB41DC00E000932F02D1CD969516CF0B
:101ED0000091A20280170895F8DBE5E68CDCF3DEC2
:101EE00041F02FDC10E079DBA9DB2DDC00E0009372
:101EF0002F0202D0999108952696899108958A9388
:101F00002497802F202F2073259525952595012F27
:101F100000710595059505950595022B086B0883BD
:101F20001295107F082F0F70012B47DD01E086DB33
:101F30006FDDCEDF11F487D001C000E024968991D7
:101F400008952497212F22952F70206E06D036DD1C
:101F500001E074DB5DDD2496089528830295007FFF
:101F60001F70102B198308952497312F307302D0DE
:101F7000206BECCF359535953595202F2071259523
:101F8000259525952595232B0895249704E9088305
:101F900009E00983DCCF9ADB802FC1DC46DC01E855
:101FA0005EDB0BDD01E04ADB36DD95DEA5CF8DDBA8
:101FB00010DD142FFCDB192F0895F9DFB0DC35DCC0
:101FC00003E84DDBFADC01E039DB25DD92CFEFDF02
:101FD0000DE1A6DC0CE1B5DF03E8088308E0F2CFF1
:101FE0002497312F3071C6DF2C62B7DFB0CF249732
:101FF00005E9088308EACDCF9A938A932497402F66
:10200000E6DBE5DF9EDBDADC05E9088308EE098321
:1020100001E014DBFDDC83DA29DB11F02BDBE1F7D7
:1020200095DB04E00E941501D2DBB5DF017011F0F1
:1020300021DBD1F7F6DBE4EAF2E0F9DBA6DF249658
:102040008991999108952497EBDA0CE008DBF6DA90
:10205000EFDADEDC0A8124960895E0DAABDABADA48
:1020600017DD0F79082B09830ADBB3DA45DF089502
:10207000D5DAA0DAAFDA0CDD0F770983882319F0FF
:10208000098100680983F0CF2697CADA93DAA2DAC9
:10209000FFDC006109830D81F7CC0E944115269772
:1020A000402E512E822F932FA42FBADA02E10883FB
:1020B00059824A828EDA03E1088399838A8300E099
:1020C00010E074DA87DA08E108831C811C7F0A2F8C
:1020D00002950F700695012B09830D810370AA0FDD
:1020E000AA0FAA0FA02BAA8374DA2696E6E00C9416
:1020F000521594DA8F708B8300E0A0DA45E08EDC15
:1021000000E09CDA45E18ADC19810A81F5DE089558
:1021100003B30F70006C08950E9444155ADCE9EA7D
:10212000F2E0A0810091A802002341F017FF02C055
:1021300011E001C010E02DDB0BE3E1DE880F991FF9
:102140008BDB1A2F08D0FDDE03E056DF01E154DF00
:10215000E3E00C945515182368DB192F0FE108955F
:102160000E94401536DCA22FB32F442EE9EAF2E09C
:1021700060800091A802002341F017FF02C011E027
:1021800001C010E006DB0BE3BADE880F991F439411
:1021900063DB0FC0182F1E7FDFDFD3DE1D91F9DA5E
:1021A00001E01EDF1D91F5DA00E01ADF01E024DF17
:1021B0000296042D4A94002369F70297162DCBDF6F
:1021C000C0DE05E019DF01E117DFE7E00C945115EF
:1021D0001123E0E3F2E02081318119F020830183B3
:1021E00002C00083318301E000932F020895002391
:1021F000E0E3F2E011F00181089500810895045FA9
:10220000A1F0045081F0025061F0035041F00A95B2
:1022100021F00A9559F413E009C017E007C01BE04C
:1022200005C017E103C01FE101C01FE2012F08959F
:10223000229711E00CE00E94D10701E0088341E001
:102240001BD006E00E9415011BD0F1F711E004E05D
:102250000E94D10703EA088300E7098341E014D014
:102260002296089507E308831BD008C008E009837D
:1022700017D030E00C2F11C050E021E030E00CC04E
:1022800000916E000023089550E020E104C009830E
:1022900041E050E02FE030E00C2F1D2F0C94F709A7
:1022A00041E050E02FE0089550E02FE030E00C2FA7
:1022B0001D2F0895239718D000E0D9DF21D010E01A
:1022C00004E019D0098340E0DFDF10E00CE013D018
:1022D00040E0D2DF23960895402E512E822F932F77
:1022E000E9EAF2E0A081B18111E005E00E94D107A6
:1022F00003E2088308950E94D10700E0088308954F
:1023000003E3088300E00983CBDFC0CF2497ECDF31
:1023100000E8ADDF01E30DD003E30BD00FD060E0A8
:1023200015D00A8101FD02C0ABDFC9F724960895DC
:1023300001E1088340E0B8DF0C94F70940E0B4DF26
:102340000E94F70900E10C94150161E002D00C94A1
:10235000040970E04FE050E02C2F3D2F2E5F3F4FDF
:102360000C2F1D2F08950E9441152497B5DF00E121
:1023700052D060D0042D007C7ADF10E006E035D02A
:1023800011F421E001C020E058D011F401E001C0B7
:1023900000E0022B032B91F05AD011F4815803C0B6
:1023A00060D011F481509F4F442455244A165B0697
:1023B00048F43BD00E94F7091DD0F8CF5AD05FD027
:1023C0000E94F7092ED007E321D005E3B2DF07E32F
:1023D000B0DFB4DF60E0BADF0A8101FD02C050DF88
:1023E000C9F72496E6E00C9452150E94D107EFE657
:1023F000F0E02DC0019701E0400E00E0501E08956E
:10240000898341E051DF0E94F70902E3088300E07D
:10241000098340E090CF3BDF07E00883598241E029
:102420008ACF10E005E00C94D10740E050E028E0AE
:1024300030E028C003E00883089530E040815181F6
:10244000628173814F33504168477940089500811C
:102450001181228133813F700F3310452044394070
:1024600008951181228133810F331041284739406B
:10247000089550E00A2F1B2F43E00C946714202F7F
:10248000312F40E0082F192F08950E943F1543D0A7
:10249000422E532EE9EAF2E08081918125DF00E1AE
:1024A00032D066240EC0C6DF0A2F060DE0DE03E13F
:1024B00020D007E11ED007E324DF07E7D4DED2DE19
:1024C00063947724082F192F1695079560167106C7
:1024D00050F3C8DE05E3C7DEC5DECADE20D035DF37
:1024E0000A8101FD02C0CCDED1F72496E8E00C940D
:1024F00050150883E42DF52D01914E2E5F2E098392
:1025000041E006C001E1C3DE07E00883B98341E092
:10251000CBDE0C94F7092497A02FB12F089500E18A
:102520000C9415010E9441152297D6DE02E073DF5C
:1025300081DFA13800E0B00710F000E801C000EC36
:102540004022498295DE10E007E04FDF11F421E0E0
:1025500001C020E072DF11F401E001C000E0022BB5
:10256000032B91F074DF11F4805803C07ADF11F46B
:1025700080509F4F442455244A165B0658F455DF7B
:102580000E94950937DFF8CF74DF085F1F4F77DFB0
:102590000E94950946DF2296E6E00C9452151BD066
:1025A000912FA2DE02E012D045DF2ADF06E309D038
:1025B0008B8107E306D00B81182F2496899199917E
:1025C0000895088360E0C5DE0C94040960DE07E02E
:1025D000088399839CCF9A938A932497802F089598
:1025E0000E94431598DF822F7FDE8CDF23DFA983D3
:1025F00011D003E10BDF9CDE03E19BDE90DF60E0A6
:10260000A5DE0A8101FD02C03BDEC9F72496E4E0A5
:102610000C9454153DDE03E10883898341DE46DED8
:102620000C94F7090E94411576DF822F932F5CDE10
:1026300069DF442413C0FEDE0A2F040D18DE03E117
:1026400008835524E82FF92FE40DF51D00810FDED6
:1026500007E3E3DE07E707DE05DE43940091AB0204
:10266000401648F303E3FFDD01E3FDDD03E3FBDD9B
:1026700003E3F9DD54DF69DE0A8101FD02C000DEFB
:10268000D1F7AFCEA8DF912F2FDE03E09FDF03E06D
:10269000C3DF03E30883898340E0B4DE03E391DF13
:1026A0000B818BCF9A938A932497902F812F1CDED6
:1026B00000E4DDDD03E18CDF882371F421DE01E33A
:1026C000D2DD03E3D0DDD4DD28D03FDE0A8101FD79
:1026D00023C0D6DDD1F771CF813071F407E311DE6D
:1026E00005E3C1DDBFDDC4DD18D02FDE0A8101FDA9
:1026F00013C0C6DDD1F761CF823071F40BE301DE88
:1027000009E3B1DD0BE3AFDDB3DD07D01EDE0A81E7
:1027100001FD02C0B5DDD1F750CF0AE00C941501E0
:102720005BDFE2DD00E2098375DF03E16FDE00DEDF
:1027300003E1FFDDF2DF60E009DE0A8101FD02C096
:102740009FDDC9F72496899108958A9324971230C2
:1027500089F0002311F484E005C0113011F48CE0FD
:1027600001C080E05EDE11D0082F0263CADD836302
:10277000888305C00AD00AE3C4DD0BE3088361E067
:10278000E5DD0B8124968991089503E2088304E036
:10279000098344CF21DFA8DD69DD4CDE31DE03E3B0
:1027A000088360E0EDCF18DF9FDD60DD03E034DFFC
:1027B00006E32CDE07E3F4CF10E010BD09B908E909
:1027C0000AB910936A031093690310937C03109362
:1027D0007B030895FA93EA933A932A931A930A9300
:1027E0003FB71CB10091690303950F730093690310
:1027F00020916A0309D010833FBF09911991299153
:102800003991E991F9911895E02FF0E0E75DFC4FDF
:102810000895FA93EA932A931A930A932FB7009193
:102820007B0310917C03011769F000917C030395F1
:102830000F7000937C03E02FF0E0E559FC4F00811E
:102840000CB901C055982FBF099119912991E991AF
:10285000F99118950BD0F1F300916A0303950F736A
:1028600000936A0310E0D0DF0081089500916903AE
:1028700010916A030117089520917B0323952F700F
:1028800030917C032317E1F3E22FF0E0E559FC4F90
:10289000008320937B03559A0895E8DF11F001E04F
:1028A000089500E008950CE90DBF03E00EBFCDE1EF
:1028B000D4E00E942B01002311F00E94881500E053
:1028C0000BBF0E9444010E94BA150C94BA154A9598
:1028D0001AF0000F111FFBCF08954A951AF01695B4
:1028E0000795FBCF08954A951AF015950795FBCFEC
:1028F000089500241124EFE0001F111F001C111C7B
:102900000416150610F0041A150AEA95AAF7001F16
:10291000111F402D512D0095109508955195419509
:1029200050400895FF27552312F4F160F7DF11237B
:1029300012F4F09507D00E947914F0FD03D0F1FD58
:10294000EDCF089511950195104008954A952AF00C
:10295000000F111F221F331FF9CF089500241124E7
:1029600022243324E0E2EA9592F0001F111F221F77
:10297000331F001C111C221C331C041615062606CE
:10298000370688F3041A150A260A370AECCF001F07
:10299000111F221F331F402D512D622D732D0095C5
:1029A00010952095309508955FD0702D5DD0602DE5
:1029B0005BD0502D59D0402D57D0102C01FA54D057
:1029C000202C52D0302C0895F5DF041B10E003C0FA
:1029D000EFDF041B150B20E030E005C0E5DF041B32
:1029E000150B260B370BE0F010FC1DC03DD0402D21
:1029F0003BD0E00FF11F0417100540E02407340717
:102A000078F446F4C895002D0024E22DF32DE01B48
:102A1000F0090994E00FF11F27D0202C25D0302C8D
:102A2000E22DF32D099411F4BEF7ECCF31960EF0A0
:102A3000319650E060E070E017D0402D4B3F68F0D9
:102A400079F34F3F41F04E3F21F00ED0702D0CD066
:102A5000602D0AD0502D08D0402D041B150B260BDD
:102A6000370B11F3E8F2E2CFC89531960895FA9248
:102A7000EA92DA92CA92BA92AA929A928A927A9236
:102A80006A925A924A92BA93AA939A938A93089511
:102A9000FF84EE84DD84CC84BB84AA8499848884FA
:102AA0007F806E805D804C80BB81AA819981888106
:102AB000F0E00FB6F894CE0FDF1F0FBE089510E0C0
:102AC0000C943C1422974C2F5D2F4E5F5F4F488330
:102AD00059834C2F5D2F5A934A9360E070E04FE585
:102AE00055E10E94BD152296089520E02D9302D055
:102AF000E1F7089501501040202F212B08953BBF8E
:102B0000D895EF5FFF4F3F4F0D92F4DFC1F7089567
:102B100002E211E0402E512EE42DF52D30E03BBFB6
:102B2000D895002D24D0102DE42DF52D3296D89572
:102B3000A02D1DD0B02DE42DF52D3496D895402D27
:102B400016D0502D14D0E42FF52F302D242F252B07
:102B5000202911F0D4DF01C0C8DF07E0400E00E0FB
:102B6000501E442D552D40335140B0F208953196FA
:102B7000D895089500008895FECF0E9437152797B5
:102B80000C831D832E83488359836A837B838F88BC
:102B9000988CCC24DD2401C0BCD0BFD005E2001647
:102BA00041F00020C9F70C2D1D2D2796E2E10C9471
:102BB000481550E040E0D895002D085621F004500B
:102BC00049F441E001C051E00E2F1F2F0F5F1F4F4E
:102BD0000C831D83A2D0002D085509F442C00B5070
:102BE00049F00A9581F10B50B1F0045039F00550CD
:102BF000C1F1D2CFB1D0A080A9D0CECFADD080814D
:102C00009181A4D0E82FF92FA1908E2F9F2FAA2079
:102C100021F27FD0F7CF08E0E02E552311F44423B2
:102C200069F480E090E8A0E0B0E0552341F104E6CB
:102C3000A01692D04080518079F52EC080E090E0BF
:102C4000A0E0B0E41EC00AE0E02E552311F44423B6
:102C500019F480E197E2E7CF80E09AECAAE9BBE3C0
:102C600010C000E1E02E552311F4442319F480E054
:102C700090E1D9CF80E090E0A0E0B0E102C0442331
:102C800041F06AD040805180628073807BD00C5FBD
:102C900007C062D0408051806624772473D00E5FD5
:102CA00057D004E6A01671F4772062F45094609433
:102CB000709404464194500A600A700A2A813B814C
:102CC0000DE24ED0823000E09007A007B007B8F0C8
:102CD000481659066A067B0690F429D0F3CF495F5F
:102CE0002A813B81042F3CD043D0442E552E662EA2
:102CF000772E1DD0012B022B032B09F44ECF38D099
:102D0000402F405D4A3360F308E7A01641F7495D64
:102D1000E7CF2A813B810A2D23C0EC81FD813E81D2
:102D20003BBFD895A02C3196EC83FD830895082FE6
:102D3000192F2A2F3B2F4E2D50E060E070E00E94AB
:102D4000AE14802F912FA22FB32F08951BD00E5FAA
:102D50001F4F00831183089515D0E02FF12F0895A0
:102D6000E881F981099501E0C00E00E0D01E0895C8
:102D7000042D152D262D372D482F592F6A2F7B2FE7
:102D80000C94AE14E82DF92D0081118108950117DE
:102D900001CB0C01000000FFFFFFFFFFFFFFFFFF63
:102DA000FFFFFFFFFFFFFFFFFFFFFFFFFFFFFFFF33
:102DB000FFFFFFFFFFFFFFFFFFFFFFFFFFFFFFFF23
:102DC000FFFFFFFFFFFFFFFFFFFFFFFFFFFFFFFF13
:102DD000FFFFFFFFFFFFFFFFFFFFFFFFFFFFFFFF03
:103800003FEF3DBF33E03EBF30E030BD37E139B977
:1038100030E43BB938E13AB936E830BDCCD0A32F1B
:10382000A03719F433E5C3D0BBC0A13619F439E58C
:10383000BED0B6C0A33579F431E4B9D036E5B7D0FF
:1038400032E5B5D032E4B3D03FE4B1D03FE4AFD0FD
:1038500034E5ADD0A5C0A43729F434E6A8D030E0D3
:10386000A6D09EC0A63529F432E3A1D031E39FD083
:1038700097C0A43509F48AC0A13449F49CD0F32F31
:103880009AD0E32FEE0FFF1F3DE091D089C0A03505
:1038900019F43DE08CD084C0AC3419F43DE087D0FD
:1038A0007FC0A33739F43EE182D034E980D032E0E2
:1038B0007ED076C0A43649F4EEBBFFBBE09A0DB2D1
:1038C000EF5FFF4F302D73D06BC0A23561F4C89508
:1038D000102CEF5FFF4FC895EF5FFF4F302D67D083
:1038E000312D65D05DC0A33609F565D0F32E0E2FBE
:1038F0000F770023B9F433E037BFE89552D03FEF9C
:10390000032E132EFF93EF9310E031E037BFE895BD
:1039100032961F3311F01395F8CFEF91FF9137B71F
:1039200030FDFDCF0F2C3DE042D03AC0A33449F426
:1039300042D0132E31E037BFE89532963DE037D0C4
:103940002FC0AD3639F435E037BFE8952AD03DE0D9
:103950002ED026C0A53619F43DE029D021C0A535CA
:1039600081F4E0E0F0E000E033E037BFE89519D003
:10397000E058FF4F003711F00395F6CF3DE017D028
:103980000FC0A83709F402C0A93721F414D03DE0D4
:103990000ED006C0AB3109F403C03FE308D000C02D
:1039A0003DCF37B730FDFDCF31E137BF08955D9B87
:1039B000FECF3CB908955F9BFECF3CB10895FF93C5
:1039C000EF93E3E3F7E03197F1F7EF91FF91E150E7
:1039D000F040A9F70895FFFFFFFFFFFFFFFFFFFF84
:1039E000FFFFFFFFFFFFFFFFFFFFFFFFFFFFFFFFE7
:1039F000FFFFFFFFFFFFFFFFFFFFFFFFFFFFFFFFD7
:103A0000FFFFFFFFFFFFFFFFFFFFFFFFFFFFFFFFC6
:103A1000FFFFFFFFFFFFFFFFFFFFFFFFFFFFFFFFB6
:00000001FF
